:020000040000FA
:020000000528D1
:08000800C528831600308600B4
:100010003630850083128501860183120313850122
:1000200007309F0083160313163085008601843045
:10003000810083120313603005178100A0308B000C
:10004000D30185014E20913058206120A3006E20FD
:10005000A4007A202308BA00AE20FA304C08D10060
:100060004D08D200A0202228051485150000093073
:10007000A200000085110000000000000000000048
:1000800085150000A20B392800004E2000008515C0
:1000900000000000851100007A2008008515051475
:1000A000851C4E28051D4E280510000085110800EE
:1000B000802005148515851C5B280000851105101E
:1000C00008008F20051000000000000000008515CA
:1000D000851C682800008511051008008F2000008D
:1000E0000000051400008515851C7428000085118A
:1000F0000510080000000000851500000514080028
:10010000A2000830AB000510A20D03180514000072
:100110008515851C89288511AB0B83280800A20151
:100120000830AB0005140000031005190314A20DDC
:100130008515851C99288511AB0B9328220808008A
:10014000FA30AD00000000000000000000000000D8
:100150000000AD0BA228AC0BA02800346430B20024
:10016000BB204E08CB000A30B200BB204E08CC00AA
:100170003A08CD000800CE01CE03CE0A3208BA02FA
:100180000318BD283208BA070800D400030E8312F2
:10019000D500603081000B1105138513D3080319B6
:1001A000DF28531003308A00520800238600831290
:1001B00003138517550E8300D40E540E09005314F3
:1001C00003308A00510800238600831203130517A9
:0A01D000550E8300D40E540E0900F2
:1006000082073F3406345B344F3466346D347D34B6
:0606100007347F346F3453
:02400E00383F39
:00000001FF
